:0200000480007A
:100000009710000093800001B7CFAAAA938FBFBBBF
:1000100023A0F00137F1F1111301212223802000E8
:1000200097120000938252FFA3AF02FEB74C33F346
:10003000938C4C4FA38F92FF171400001304F4FD10
:10004000A3200400B7FFF555938F6F66A300F4015A
:10005000971500009385C57C23A00580379677F718
:100060001306868F2380C580170700001307977B30
:10007000A32F077EB71709999387A7AAA30FF77E27
:1000800097180000938888FA371911111309C910BD
:10009000B72922229389C92C373A3333130ABA3B42
:1000A000B74A4444938ABA40375B5555130BEB5E0D
:1000B000B76B6666938BEB60377C7777130CDC70DD
:1000C000B79C8888938CDC8D37AD9999130D0D9F63
:1000D000B7BDAAAA938D0DA037CEBBBB130EFEBF32
:1000E000B7DECCCC938EFEC0238E28FFA38E38FFC4
:1000F000238F48FFA38F58FF23806801A3807801D6
:1001000023818801A38198012382A801A382B801D9
:100110002383C801A383D801171B0000130B8BF1A5
:10012000B74065879380103223201B00375034126C
:100130001300806723000B00971A0000938A8AEC53
:1001400083A00A0023A00000B73922119389493403
:1001500083AB0A0023803B01971B0000938BCBEA03
:10016000171C0000130C8CED23200C0083AC0B003B
:1001700023009C01171D0000130D8DEC23200D00A2
:10018000B73C5476938C0C2123009D01930C000006
:10019000171E0000130E0EEB23200E00B7DDAB89F7
:1001A000938DFDDE2300BE01130ECEFF971E0000CF
:1001B000938E8EE923A00E0023A20E00B76D721459
:1001C000938D6D832380BE0103AF0E002382EE0169
:1001D000971000009380C0E723A0000037513896A5
:1001E00013011120B751812593813196238020007E
:1001F00023803000171500001305C5E19715000096
:10020000938545E5370610F01306C6F26306B5027E
:100210008326C5002320D600832685002320D60010
:10022000832645002320D600832605002320D60000
:10023000130505016FF09FFD370510F0130505F25A
:040240002320050072
:1010000034100080F0DEBC9A0000000000000000F8
:10101000FFFFFFFFFFFFFFFFFFFFFFFFFFFFFFFFE0
:10102000FFFFFFFFFFFFFFFFFFFFFFFFFFFFFFFFD0
:10103000FFFFFFFFFFFFFFFFFFFFFFFFFFFFFFFFC0
:10104000FFFFFFFFFFFFFFFFFFFFFFFFFFFFFFFFB0
:040000058000000077
:00000001FF
